:020000040801F1
:1000000000000220DD410108B12B0108B52B0108D9
:10001000B92B0108BD2B0108C12B0108000000000D
:10002000000000000000000000000000C52B0108D7
:10003000C92B010800000000CD2B0108D12B0108BD
:100040002D4201082D4201082D4201082D420108D0
:100050002D4201082D4201082D4201082D420108C0
:100060002D4201082D4201082D4201082D420108B0
:100070002D4201082D4201082D4201082D420108A0
:100080002D4201082D4201082D4201082D42010890
:100090002D4201082D4201082D4201082D42010880
:1000A0002D4201082D4201082D4201082D42010870
:1000B0002D4201082D4201082D4201082D42010860
:1000C0002D4201082D4201082D4201082D42010850
:1000D0002D420108E12B0108ED2B01082D420108FA
:1000E0002D4201082D4201082D4201082D42010830
:1000F0002D4201082D4201082D4201082D42010820
:100100002D4201082D4201082D4201082D4201080F
:10011000F92B01082D4201082D4201082D4201084A
:100120002D4201082D4201082D4201082D420108EF
:100130002D4201082D4201082D4201082D420108DF
:100140002D4201082D4201082D4201082D420108CF
:100150002D4201082D4201082D4201082D420108BF
:100160002D4201082D4201082D4201082D420108AF
:100170002D4201082D4201082D4201080000000017
:080180002D4201082D42010887
:10019000044B05481B1A062B02D9044B03B1184720
:1001A000704700BF9F0000209C000020000000005E
:1001B00005490648091A891001EBD171491002D08E
:1001C000034B03B1184770479C0000209C0000209F
:1001D0000000000010B5064C237843B9FFF7D8FFA4
:1001E000044B13B10448AFF300800123237010BD0A
:1001F0009C000020000000003042010808B5084BB8
:100200001BB108490848AFF300800848036813B9D8
:10021000BDE80840CCE7064B002BF9D09847F7E73C
:1002200000000000A0000020304201089C000020D7
:100230000000000070B50F4E0F4D761BB61018BFB2
:10024000002405D0013455F8043B9847A642F9D163
:100250000A4E0B4D761B03F0EBFFB61018BF0024BF
:1002600006D0013455F8043B9847A642F9D170BD39
:1002700070BD00BF2043010820430108244301084A
:100280002043010870B4860746D0541E002A41D08E
:10029000CAB2034602E014F1FF343BD303F8012B4A
:1002A0009D07F8D1032C2ED9CDB245EA05250F2C98
:1002B00045EA054519D903F110022646103E0F2ED6
:1002C00042F8105C42F80C5C42F8085C42F8045CAE
:1002D00002F11002F2D8A4F1100222F00F0204F091
:1002E0000F041032032C13440DD91E462246043A43
:1002F000032A46F8045BFAD8221F22F003020432D4
:10030000134404F003042CB1C9B21C4403F8011BCC
:100310009C42FBD170BC704714460346C2E700BF45
:100320000EB410B5044683B018B183690BB900F060
:100330001FF906A803460190059AA168204600F01F
:1003400023FA03B0BDE8104003B070470FB410B5F6
:100350000A4B1C6882B024B1A36913B9204600F08F
:1003600007F905A803460190049AA168204600F009
:100370000BFA02B0BDE8104004B070470000002046
:1003800000207047014900F039B900BFB9110108D8
:100390000020704770B54A1E682505FB02F50E4621
:1003A00005F1740100F054F9044640B100210C300D
:1003B000666005F168022160A060FFF763FF2046D8
:1003C00070BD00BF204B70B51D68AB6906465BB3BE
:1003D00048356B68AC68013B05D521E0013B5A1CF0
:1003E00004F168041CD0B4F90C20002AF6D10025D1
:1003F0004FF6FF720123E281A38165662560A56047
:10040000656025616561A5612946082204F15C00EB
:10041000FFF738FF6563A563A564E564204670BDFA
:10042000286828B10546D4E7284600F00FF8CFE742
:1004300004213046FFF7AEFF28600028F2D10C23DC
:1004400004463360EAE700BF484201083D4B3E499D
:100450001A682DE9F04F90424FF000038364C364A3
:10046000036508BF012383B008BF8361816207462B
:10047000FFF7A8FF78603846FFF7A4FFB86038465A
:10048000FFF7A0FF7D68F86000240423AB812C6097
:100490006C60AC606C66EC812C616C61AC61214677
:1004A00005F15C000822FFF7EDFEBE68DFF89CB0A6
:1004B000DFF89CA0DFF89C90DFF89C80C5F824B0A2
:1004C00001230922C5F828A0C5F82C90C5F8308072
:1004D0002D622146F381B28134607460B460746629
:1004E00034617461B46106F15C0008220193FFF786
:1004F000C9FEFD68366212200222C6F824B0C6F892
:1005000028A0C6F82C90C6F830802146A881EA8140
:100510002C606C60AC606C662C616C61AC6105F148
:100520005C000822FFF7AEFE019B2D62C5F824B0E7
:10053000C5F828A0C5F82C90C5F83080BB6103B081
:10054000BDE8F08F4842010885030108FD0D010850
:10055000250E0108610E0108810E0108024B0349B6
:10056000186800F04BB800BF48420108B9110108F3
:10057000836903B96AE77047704700BF704700BFDF
:10058000704700BF704700BF024B0349186800F076
:100590000FB800BF0000002091030108024B03497F
:1005A000186800F005B800BF0000002081030108B2
:1005B0002DE9F04110F148071BD0884600267D68E0
:1005C000BC68013D0FD4A389012B05F1FF3506D985
:1005D000B4F90E300133204601D0C04706436B1CEE
:1005E00004F16804EFD13F68002FE8D13046BDE840
:1005F000F0813E463046BDE8F08100BF2DE9F8436A
:1006000010F148071FD0884606464FF000097D6864
:10061000BC68013D11D4A389012B05F1FF3508D930
:10062000B4F90E3001332146304602D0C04749EAC2
:1006300000096B1C04F16804EDD13F68002FE6D17E
:100640004846BDE8F883B9464846BDE8F88300BF90
:1006500070B5CC1C24F0030408340C2C38BF0C24D7
:10066000002C06463BDBA14239D8274D296851B101
:100670000A68121B04D436E01A68121B1AD51946F0
:100680004B68002BF8D16968002937D021463046E5
:1006900000F0A2FB431C22D0C31C23F00305A84298
:1006A00005D0291A304600F097FB013017D02C6096
:1006B0002B4604E00B2A0DD91A6013441C6003F189
:1006C0000B0020F007001A1D821A02D051429950E7
:1006D00070BD70BD8B420ED05A684A60EFE70C23A4
:1006E0003360002070BD0B2A03D84A680B462A608D
:1006F000E5E70B46E0E70A460B46F8E7304600F030
:100700006BFB6860C2E700BFB80000209368013B44
:10071000002B10B4936008DBCCB21368581C106037
:10072000197020465DF8044B70479469A34202DBC0
:10073000CCB20A2CF1D15DF8044B00F0A5BB00BF90
:1007400093B1F8B514460F460646D51801E0AC4201
:1007500008D03A4614F8011B3046FFF7D7FF431C78
:10076000F5D1F8BD0020F8BD00207047936810B5A2
:10077000144613B95360184610BD00F061FD002304
:10078000A360636010BD00BF2DE9F04F9DB08946A6
:1007900014460393824618B18369002B00F00A8146
:1007A0008A4B994500F00C81894B994500F00B81EB
:1007B000884B994508BFDAF80C90B9F80C30180747
:1007C00040F1EE80D9F81030002B00F0E9803023A2
:1007D0008DF82A302378804E0021202209918DF84F
:1007E00029200127002B00F08480252B254603D1EA
:1007F00017E0252B00F0858015F8013F002BF8D17C
:10080000B5EB040B75D022465B4649465046FFF7D0
:1008100097FF01306DD0099B2A785B440993002A29
:1008200067D000234FF0FF320135049307930693FE
:100830008DF853301A93059204E0049A07FA03F3F3
:100840001343049329780522304600F0F9FE2C4624
:10085000831B01350028F0D1049BD90644BF202218
:100860008DF8532021781A0744BF2B228DF853208E
:100870002A2969D0A1F13002092A0BD8079B14F864
:10088000011F03EB830302EB4303A1F13002092AAA
:10089000F5D907932E293FD0504D0322284600F06A
:1008A000CFFE38B1049B401B402202FA00F0034304
:1008B0000134049321784A488DF828100622013427
:1008C00000F0BEFE002849D0464BF3B103AB0093C5
:1008D0004A46454B04A95046AFF300808046B8F124
:1008E000FF3F06D0099B434409932378002B7FF4F4
:1008F0007CAFB9F80C305B0659D409981DB0BDE83F
:10090000F08FB5EB040B8CD07DE7039B073323F00E
:10091000070308330393E5E761782A2904F101000E
:1009200026D0A1F130020023092A05930446B3D84A
:1009300014F8011F03EB830302EB4303A1F1300220
:10094000092AF5D90593A7E7039A1168043200290B
:1009500003921FDB0791617801349BE703AB00939F
:100960004A46214B04A9504600F0E6F88046B6E717
:10097000039B1A680592002A03F104030393B8BF8E
:100980004FF0FF3204F10203AEBFA178A1780592C7
:100990001C4681E7494243F0020307910493DAE7DA
:1009A0004946504600F0E8FA00283FF410AF4FF0F7
:1009B000FF30A3E7FFF7DCFD044B99457FF4F4AE6D
:1009C000DAF80490F9E6DAF80890F6E68C420108C5
:1009D0006C4201084C420108E4420108EC42010863
:1009E000F0420108000000004107010810B4044C67
:1009F00013460A46014620685DF8044BFFF7C4BE63
:100A0000000000202DE9F0470C4691460A698968EC
:100A1000DDF820808A42B8BF0A46C9F8002094F861
:100A2000431006461F4611B10132C9F80020236861
:100A300099065DD5D9F800200232C9F80020236854
:100A400013F0060F19461DD1E1688A1A002AD8BF93
:100A5000194617DD04F1190A002505E0E368D9F805
:100A600000209B1AAB420CDD01235246394630462A
:100A7000C047013005F10105F0D14FF0FF30BDE86E
:100A8000F087216894F84330003318BF01238A06A9
:100A90000AD5E1185A1C302081F84300224494F80A
:100AA000451082F84310023304F1430239463046C0
:100AB000C0470130E1D0236803F00603042B29D09E
:100AC000A36822699342C8BF4FF0000930DD9B1A2A
:100AD00099441A34002501E04D4529D001232246CE
:100AE00039463046C047013005F10105F4D1C4E76D
:100AF00013F0060F08D1E168D9F800208A1A002AFD
:100B0000D8BF1946A6DCBDE794F84330003318BFC0
:100B10000123C9E7D9F80010E068A3682269A0EBB7
:100B20000109934229EAE979D1DCB9F1000FD0D16A
:100B30000020BDE8F08700BF2DE9F0430C46097E98
:100B400085B06E29064617460C98984604F1430C6A
:100B500055D00FD8632900F01B8100F2D680002900
:100B60005CD0582940F0E88084F845102268DFF80E
:100B700060E213E0732900F0FD8000F289806F29A4
:100B800000F0E480702940F0D780226842F0200213
:100B900022607823DFF83CE284F8453003681506CC
:100BA00003F1040100F1FF8055064BBF1B881B6851
:100BB00001600160D00744BF42F020022260002B98
:100BC00040F09580226822F020022260102100224D
:100BD00084F843206068A0600028C0F28D802268FD
:100BE00022F004022260002B67D1002840F08680AA
:100BF000654608296FD0ACEB0503236111E023683B
:100C00001A0600F1D38013F0400F0368626903F104
:100C1000040101601B6814BF1A801A600023654636
:100C20002361CDF800803B4603AA21463046FFF7FA
:100C3000E9FE013021D02A46236939463046C047B3
:100C400001301AD02368E06813F0020F039B19D01B
:100C5000C21A002A16DD04F11909002504E0E06833
:100C6000039BC21AAA420DDD01234A46394630468B
:100C7000C047013005F10105F1D14FF0FF3005B05B
:100C8000BDE8F0839842B8BF184605B0BDE8F083D0
:100C900075295BD078294FD122687AE76168A16015
:100CA0002D200029C3F1000384F8430021DB22F04A
:100CB0000402DFF81CE122600A216546B3FBF1F271
:100CC00001FB123013461EF8002005F8012D002B01
:100CD000F4D108298FD12368D9078CD5626823699C
:100CE0009A4288DC302305F8013C013D83E710215E
:100CF0006DE7DFF8DCE00A21002BDED19EF8003042
:100D000084F8423004F1420573E7642901D069296F
:100D100012D122680368150603F1040152D4550666
:100D20004BBFB3F900301B6801600160002BB5DBDD
:100D3000DFF89CE00A214DE7012384F8421023618B
:100D400004F14205002384F843306AE723681A0659
:100D500033D413F0400F036803F1040215BF1B885E
:100D60001B68026002606F2914BF0A210821DFF8A6
:100D700060E02CE703686268191D01601D680021AE
:100D8000284600F05DFC00B3401B60602061D9E79D
:100D900003681A68191D0123016004F1420584F8F3
:100DA00042202361CEE701601B6803E703686269A4
:100DB000191D01601B681A6030E703681A1D026084
:100DC0001B68D0E701601B68B0E76068DEE700BF22
:100DD000F84201080C43010838B5074C00230546CA
:100DE0000846236000F058FE431C00D038BD23683D
:100DF000002BFBD02B6038BD1402002010B50C4630
:100E0000B1F90E1000F0DAFD002803DB636D034436
:100E1000636510BDA38923F48053A38110BD00BF77
:100E2000002070472DE9F0411646B1F90C201F460D
:100E3000D3050C46054607D500220223B1F90E1052
:100E400000F076FBB4F90C20B4F90E1022F48052B5
:100E5000A2813B4632462846BDE8F04100F076B814
:100E600010B50C46B1F90E1000F062FBA389421CCC
:100E70000EBF23F4805343F480536065A38110BDFB
:100E8000B1F90E1000F0F2B8F8B50D46144606465A
:100E900010B18369002B42D0254B9C4244D0254B96
:100EA0009C4243D0244B9C4208BFF468A389A269AA
:100EB000A2601A0722D5236903B322686169D31A95
:100EC000EDB28B422F4621DA0133A168501C013963
:100ED000A1602060157062699A4206D0A389DB0781
:100EE00001D50A2D01D03846F8BD2146304600F024
:100EF00063F90028F7D04FF0FF37F4E7214630467A
:100F000000F03AF80028F6D12369D6E721463046AA
:100F100000F052F90028EED122680123D5E7FFF74F
:100F200027FB034B9C42BAD17468BFE7B468BDE7A6
:100F30008C4201086C4201084C420108024B0A46EF
:100F400001461868FFF7A0BF0000002070B50D46ED
:100F5000084C114606461A4628460023236001F035
:100F6000C3F9431C00D070BD2368002BFBD0336055
:100F700070BD00BF14020020384B70B51D680646D6
:100F80000C4615B1AB69002B42D0354B9C4245D085
:100F9000344B9C4258D0344B9C4208BFEC68B4F9A7
:100FA0000C2093B219070CD52069A8B113F00102E7
:100FB0001ED0636900225B42A361A260F0B10020F1
:100FC00070BDDD0642D558072AD4206942F00803D7
:100FD000A3819BB20028E9D103F42072B2F5007F0F
:100FE000E4D03046214600F0E7FAA3892069DDE726
:100FF000990758BF6269A2600028E0D1B4F90C30AB
:101000001A06DDD543F04003A3814FF0FF3070BDD9
:101010002846FFF7ADFA124B9C42B9D16C68BEE787
:10102000616B51B104F14403994204D0304600F0A1
:1010300055FCB4F90C20002363630023206963602E
:1010400022F024022060C1E7AC68A8E742F0400229
:10105000092333604FF0FF30A28170BD00000020F3
:101060008C4201086C4201084C42010838B5074C1B
:10107000002305460846236000F0E6FC431C00D030
:1010800038BD2368002BFBD02B6038BD1402002034
:101090008B891A072DE9F0410D46804633D44A6802
:1010A000002A67DDEC6A002C45D00022D8F80060E9
:1010B000C8F8002013F4805260D06A6D5F0705D530
:1010C00069686B6B521A0BB12B6CD21A0023296A18
:1010D0004046A047441C39D0AB892A692A60DB040A
:1010E0004FF000026A6043D4696BC8F8006011B326
:1010F00005F14403994202D0404600F0EFFB002086
:101100006863BDE8F0810E69AEB10C680E609807A7
:101110000CBF4B690023A41B8B600AE023463246B8
:10112000AF6A296A4046B8470028A4EB0004064489
:1011300004DD002CF2DC0020BDE8F081AB8943F037
:101140004003AB814FF0FF30BDE8F081D8F80020BC
:101150001D2AF3D8174BD340DB4313F00103EDD125
:10116000A9892C696B60C9042C60BDD5002ABBD14C
:101170006865B9E70A6C002A94DCDCE70123296A78
:101180004046A047431C024602D0AB89EC6A95E773
:10119000D8F80030002BF8D01D2B01D0162B02D12F
:1011A000C8F80060C7E7AB8943F04003AB81BDE8F6
:1011B000F08100BF010040200B6933B310B5044635
:1011C00082B008B18369ABB1114B994219D0114B70
:1011D000994218D0104B994208BFE168B1F90C3020
:1011E00013B9002002B010BD204602B0BDE8104087
:1011F000FFF74EBF0191FFF7BBF90199044B9942EC
:10120000E5D16168EAE7A168E8E70020704700BF20
:101210008C4201086C4201084C42010820B1054B88
:1012200001461868FFF7C8BF034B04491868FFF769
:10123000E5B900BF0000002048420108B9110108CB
:101240009368002B73D02DE9F04F8B8983B00C4647
:1012500019070090164626D5226922B313F0020022
:1012600035682CD04FF00009B04FC846B246B8459B
:1012700043464A4628BF3B460098B8F1000F50D07D
:10128000216AA66AB047002858DDDAF808301B1A30
:101290008144A8EB0008CAF80830002BE7D10020F1
:1012A00003B0BDE8F08F21460098FFF765FE0028E7
:1012B00040F03381A389356813F00200D2D113F0D6
:1012C000010945D14F46019637B39A05D4F80880F5
:1012D00040F183804745C346C0F0AB8013F4906F64
:1012E00040F0AC802068BA465A46494600F092FA6F
:1012F000A2682368A2EB08025B44A2602360019A03
:101300009368A3EB0A03D144A7EB0A079360002B71
:10131000C5D0A389002FD8D1D5F800906F680835C3
:10132000D2E7D5F80090D5F8048008359FE7002073
:10133000704721460098FFF73FFF70B3B4F90C30B7
:1013400043F040034FF0FF30A38103B0BDE8F08FBE
:10135000814633464E46A8469A464D464EB380B324
:10136000206823696269B145CB4628BFB3469842DD
:101370005F4604D9A36813449B4500F3A6809345B8
:101380004BDB1346A76A216A00982A46B847071E16
:10139000D4DDB9EB0709CCD00120DAF80830DB1B2B
:1013A0003D44F61BCAF80830002B3FF478AF002EFE
:1013B000D5D108F1080313E9600098460833002EE0
:1013C000F9D032460A21284600F03AF9002800F008
:1013D000A1800130A0EB0509C2E72068236998428B
:1013E00002D863699F425DD2B84528BFB8464246DD
:1013F000494600F00FFAA3682268A3EB08034244B1
:10140000A36022600BB1C24679E721460098FFF73E
:10141000D3FE002892D1C24671E75A46294600F011
:10142000F9F9A2682368A2EB0B025B44A260236077
:10143000AFE72068B846BA46BB4655E76269206800
:10144000216902EB4208A0EB010A08EBD8780AF107
:1014500001004FEA680838444045424684BF804650
:1014600042465B0544D511460098FFF7F1F88346E4
:10147000002855D05246216900F032F9A38923F49F
:10148000906343F08003A3810BEB0A00A8EB0A03EF
:10149000C4F810B0C4F814802060A360B846BA46FF
:1014A000BB4621E76FF00041B94228BF39464A46A2
:1014B00091FBF3F10098A66A03FB01F3216AB047A0
:1014C000B0F1000A3FF71BAF38E71A4629460193EF
:1014D00000F0A0F92268019B00981A44226021467E
:1014E000FFF76AFE019B00287FF428AF1F4650E7F4
:1014F000009800F03BFA83460028C5D1009D216981
:10150000284600F0EBF9B4F90C300C2223F08003EC
:101510002A6015E706F1010922E74FF0FF30BFE628
:10152000009A0C231360B4F90C3009E700FCFF7F2C
:1015300070B50D46084C114606461A46284600234B
:10154000236000F099FA431C00D070BD2368002B83
:10155000FBD0336070BD00BF1402002070B50C4694
:10156000B1F90E10002990B015461E4613DB01AAF2
:1015700000F03AFA00280EDB029A02F47042A2F55B
:101580000052B2FA82F252094FF4806300203260B6
:101590002B6010B070BDA38900221B06326004D5F9
:1015A000402300202B6010B070BD4FF480630020FA
:1015B0002B6010B070BD00BF8A8992070B4606D51C
:1015C00001F1470201211A601A6159617047F0B5B3
:1015D00083B001AB6A460C460546FFF7BFFF009992
:1015E00006462846FFF734F8B4F90C30D0B1019A1A
:1015F000124F0099AF6243F08003A3812060206105
:1016000061611AB93343A38103B0F0BD2846B4F930
:101610000E1000F0FDF9B4F90C300028F2D043F0C0
:101620000103EFE79A05EFD404F1470243F0020308
:101630000121A381226022616161E5E78503010840
:1016400001F0FF01102A2BDB10F0070F08D010F873
:10165000013B013A8B422DD010F0070F42B3F6D177
:10166000F0B441EA012141EA014122F007047FF090
:1016700000070023F0E80256083C85EA010586EAE7
:10168000010685FA47F5A3FA87F586FA47F6A5FA23
:1016900087F68EB9EED1F0BC01F0FF0102F007022F
:1016A00032B110F8013B013A83EA010313B1F8D1DA
:1016B0000020704701387047002D06BF35460338BB
:1016C000073815F0010F07D1013015F4807F02BFF4
:1016D000013015F4C03F0130F0BC0138704700BF45
:1016E000844641EA000313F003036DD1403A41D32D
:1016F00051F8043B40F8043B51F8043B40F8043BEC
:1017000051F8043B40F8043B51F8043B40F8043BDB
:1017100051F8043B40F8043B51F8043B40F8043BCB
:1017200051F8043B40F8043B51F8043B40F8043BBB
:1017300051F8043B40F8043B51F8043B40F8043BAB
:1017400051F8043B40F8043B51F8043B40F8043B9B
:1017500051F8043B40F8043B51F8043B40F8043B8B
:1017600051F8043B40F8043B51F8043B40F8043B7B
:10177000403ABDD2303211D351F8043B40F8043B1B
:1017800051F8043B40F8043B51F8043B40F8043B5B
:1017900051F8043B40F8043B103AEDD20C3205D32B
:1017A00051F8043B40F8043B043AF9D2043208D023
:1017B000D2071CBF11F8013B00F8013B01D30B8895
:1017C00003806046704700BF082A13D38B078DD073
:1017D00010F003038AD0C3F10403D21ADB071CBF45
:1017E00011F8013B00F8013B80D331F8023B20F8AF
:1017F000023B7BE7043AD9D3013A11F8013B00F8E8
:10180000013BF9D20B7803704B7843708B7883706F
:10181000604670478842F0B50DD98B1898420AD2BD
:101820008418002A51D0224613F8014D02F8014DC8
:101830009942F9D1F0BD0F2A48D941EA00039B072C
:1018400046D100F1100401F11003154653F8106C55
:1018500044F8106C53F80C6C44F80C6C53F8086C9A
:1018600044F8086C103D53F8046C44F8046C0F2DD8
:1018700003F1100304F11004E8D8A2F1100323F0DF
:101880000F0302F00F0E1033BEF1030F194403448F
:1018900021D91E1F0D467446043C55F8047B46F8BA
:1018A000047F032CF8D8AEF1040424F003040434BC
:1018B0002144234402F0030262B1013B0A4411F8BF
:1018C000014B03F8014F8A42F9D1F0BD0346F3E71B
:1018D0000346F2E7F0BD7246EEE700BF91B151F862
:1018E000043C0439002BB8BFC9181F4B1A68FAB161
:1018F0008A4230B40AD908680C18A24226D04A603D
:10190000196030BC70478B4203D81A465368002BCD
:10191000F9D1146815198D420DD006D808680C1835
:101920009C4219D04B605160EBE70C230360E8E761
:101930004A601960704709680C4411199942146093
:10194000DFD10ACB0C4453601460DAE714685268A4
:101950004A6020440860D3E71C685B684B60204401
:1019600008605160CDE700BFB8000020F8B514460C
:10197000F9B1C2B106460D4600F05CF8844201D8C8
:101980002846F8BD21463046FEF762FE074670B194
:1019900022462946FFF7A4FE294630463D46FFF77A
:1019A0009DFF2846F8BDFFF799FF2546E8E7054665
:1019B000E6E71146BDE8F840FEF74ABE70B50D46B1
:1019C000084C114606461A4628460023236000F0BC
:1019D0005BF8431C00D070BD2368002BFBD0336044
:1019E00070BD00BF1402002038B50B46074C0546F9
:1019F000114618460023236000F02EF8431C00D047
:101A000038BD2368002BFBD02B6038BD14020020AA
:101A100038B5074C002305460846236000F024F83B
:101A2000431C00D038BD2368002BFBD02B6038BD91
:101A30001402002051F8040C0028A0F10400BCBFDF
:101A40000B58C018704700BF024B58221A604FF065
:101A5000FF30704714020020024B58221A604FF0EA
:101A6000FF30704714020020024B58221A600020F9
:101A7000704700BF14020020024B58221A604FF03A
:101A8000FF30704714020020024B58221A604FF0BA
:101A9000FF30704714020020044A05491368002BE8
:101AA00008BF0B461844106018467047C00000205D
:101AB0001802002081F0004102E000BF83F00043E3
:101AC00030B54FEA41044FEA430594EA050F08BFD9
:101AD00090EA020F1FBF54EA000C55EA020C7FEA9D
:101AE000645C7FEA655C00F0E2804FEA5454D4EB1A
:101AF0005555B8BF6D420CDD2C4480EA020281EAE4
:101B0000030382EA000083EA010180EA020281EA1B
:101B10000303362D88BF30BD11F0004F4FEA01316D
:101B20004FF4801C4CEA113102D0404261EB41017C
:101B300013F0004F4FEA03334CEA133302D0524202
:101B400063EB430394EA050F00F0A780A4F10104BE
:101B5000D5F1200E0DDB02FA0EFC22FA05F28018F8
:101B600041F1000103FA0EF2801843FA05F35941DE
:101B70000EE0A5F120050EF1200E012A03FA0EFC5D
:101B800028BF4CF0020C43FA05F3C01851EBE37187
:101B900001F0004507D54FF0000EDCF1000C7EEBA4
:101BA00000006EEB0101B1F5801F1BD3B1F5001FE2
:101BB0000CD349085FEA30004FEA3C0C04F1010401
:101BC0004FEA445212F5800F80F09A80BCF1004F2A
:101BD00008BF5FEA500C50F1000041EB045141EAAC
:101BE000050130BD5FEA4C0C404141EB010111F4AD
:101BF000801FA4F10104E9D191F0000F04BF014658
:101C00000020B1FA81F308BF2033A3F10B03B3F135
:101C100020020CDA0C3208DD02F1140CC2F10C02C5
:101C200001FA0CF021FA02F10CE002F11402D8BF23
:101C3000C2F1200C01FA02F120FA0CFCDCBF41EAEF
:101C40000C019040E41AA2BF01EB0451294330BDBE
:101C50006FEA04041F3C1CDA0C340EDC04F114049B
:101C6000C4F1200220FA04F001FA02F340EA030072
:101C700021FA04F345EA030130BDC4F10C04C4F1B8
:101C8000200220FA02F001FA04F340EA0300294698
:101C900030BD21FA04F0294630BD94F0000F83F4E2
:101CA000801306BF81F480110134013D4EE77FEAC5
:101CB000645C18BF7FEA655C29D094EA050F08BF11
:101CC00090EA020F05D054EA000C04BF19461046F2
:101CD00030BD91EA030F1EBF0021002030BD5FEA36
:101CE000545C05D14000494128BF41F0004130BD5E
:101CF00014F580043CBF01F5801130BD01F00045B2
:101D000045F0FE4141F470014FF0000030BD7FEA24
:101D1000645C1ABF194610467FEA655C1CBF0B461F
:101D2000024650EA013406BF52EA033591EA030F36
:101D300041F4002130BD00BF90F0000F04BF00212E
:101D4000704730B54FF4806404F132044FF0000561
:101D50004FF0000150E700BF90F0000F04BF0021DA
:101D6000704730B54FF4806404F1320410F0004540
:101D700048BF40424FF000013EE700BF42004FEA3B
:101D8000E2014FEA31014FEA02701FBF12F07F43B8
:101D900093F07F4F81F06051704792F0000F14BFB5
:101DA00093F07F4F704730B54FF4607401F00045F9
:101DB00021F0004120E700BF50EA010208BF704750
:101DC00030B54FF000050AE050EA010208BF704745
:101DD00030B511F0004502D5404261EB41014FF4AE
:101DE000806404F132045FEA915C3FF4DCAE4FF0B2
:101DF00003025FEADC0C18BF03325FEADC0C18BF99
:101E0000033202EBDC02C2F1200300FA03FC20FAE9
:101E100002F001FA03FE40EA0E0021FA02F1144436
:101E2000C1E600BF70B54FF0FF0C4CF4E06C1CEA4B
:101E300011541DBF1CEA135594EA0C0F95EA0C0FC0
:101E400000F0DEF82C4481EA030621EA4C5123EA33
:101E50004C5350EA013518BF52EA033541F4801162
:101E600043F4801338D0A0FB02CE4FF00005E1FB15
:101E700002E506F00042E0FB03E54FF00006E1FB5F
:101E800003569CF0000F18BF4EF0010EA4F1FF04A2
:101E9000B6F5007F64F5407404D25FEA4E0E6D41E2
:101EA00046EB060642EAC62141EA55514FEAC520F3
:101EB00040EA5E504FEACE2EB4F1FD0C88BFBCF56F
:101EC000E06F1ED8BEF1004F08BF5FEA500E50F120
:101ED000000041EB045170BD06F0004646EA0101E6
:101EE00040EA020081EA0301B4EB5C04C2BFD4EB18
:101EF0000C0541EA045170BD41F480114FF0000E11
:101F0000013C00F3AB8014F1360FDEBF002001F07E
:101F1000004170BDC4F10004203C35DA0C341BDCF8
:101F200004F11404C4F1200500FA05F320FA04F0CA
:101F300001FA05F240EA020001F0004221F00041FE
:101F400010EBD37021FA04F642EB06015EEA430E71
:101F500008BF20EAD37070BDC4F10C04C4F12005A1
:101F600000FA04F320FA05F001FA04F240EA020054
:101F700001F0004110EBD37041F100015EEA430E25
:101F800008BF20EAD37070BDC4F1200500FA05F245
:101F90004EEA020E20FA04F301FA05F243EA0203C4
:101FA00021FA04F001F0004121FA04F220EA0200D3
:101FB00000EBD3705EEA430E08BF20EAD37070BD19
:101FC00094F0000F0FD101F00046400041EB0101F9
:101FD00011F4801F08BF013CF7D041EA060195F0DB
:101FE000000F18BF704703F00046520043EB030395
:101FF00013F4801F08BF013DF7D043EA0603704782
:1020000094EA0C0F0CEA135518BF95EA0C0F0CD08C
:1020100050EA410618BF52EA4306D1D181EA0301D2
:1020200001F000414FF0000070BD50EA410606BFCC
:102030001046194652EA430619D094EA0C0F02D111
:1020400050EA013613D195EA0C0F05D152EA033656
:102050001CBF104619460AD181EA030101F0004174
:1020600041F0FE4141F470014FF0000070BD41F0BD
:10207000FE4141F4780170BD70B54FF0FF0C4CF497
:10208000E06C1CEA11541DBF1CEA135594EA0C0FB6
:1020900095EA0C0F00F0A7F8A4EB050481EA030E03
:1020A00052EA03354FEA013100F088804FEA0333EA
:1020B0004FF0805545EA131343EA12634FEA0222B8
:1020C00045EA111545EA10654FEA00260EF0004179
:1020D0009D4208BF964244F1FD0404F5407402D2CB
:1020E0005B084FEA3202B61A65EB03055B084FEA5C
:1020F00032024FF480104FF4002CB6EB020E75EB59
:10210000030E22BFB61A754640EA0C005B084FEA80
:102110003202B6EB020E75EB030E22BFB61A7546FD
:1021200040EA5C005B084FEA3202B6EB020E75EB48
:10213000030E22BFB61A754640EA9C005B084FEAC0
:102140003202B6EB020E75EB030E22BFB61A7546CD
:1021500040EADC0055EA060E18D04FEA051545EABC
:1021600016754FEA06164FEAC30343EA52734FEA65
:10217000C2025FEA1C1CC0D111F4801F0BD141EADE
:1021800000014FF000004FF0004CB6E711F4801F43
:1021900004BF01430020B4F1FD0C88BFBCF5E06F23
:1021A0003FF6AFAEB5EB030C04BFB6EB020C5FEA33
:1021B000500C50F1000041EB045170BD0EF0004E88
:1021C0004EEA113114EB5C04C2BFD4EB0C0541EABA
:1021D000045170BD41F480114FF0000E013C90E6B7
:1021E00045EA060E8DE60CEA135594EA0C0F08BF7B
:1021F00095EA0C0F3FF43BAF94EA0C0F0AD150EA7A
:1022000001347FF434AF95EA0C0F7FF425AF10460C
:1022100019462CE795EA0C0F06D152EA03353FF434
:10222000FDAE1046194622E750EA410618BF52EAB1
:1022300043067FF4C5AE50EA41047FF40DAF52EA85
:1022400043057FF4EBAE12E74FEA4102B2F1E043FF
:1022500024BFB3F5001CDCF1FE5C0DD901F0004C8D
:102260004FEAC0024CEA5070B2F1004F40EB8300DD
:1022700008BF20F00100704711F0804F21D113F109
:102280003872BCBF01F00040704741F480114FEA42
:102290005252C2F11802C2F1200C10FA0CF320FACB
:1022A00002F018BF40F001004FEAC1234FEAD323E8
:1022B00003FA0CFC40EA0C0023FA02F34FEA430352
:1022C000CCE77FEA625307D150EA01331EBF4FF0DB
:1022D000FE4040F44000704701F0004040F0FE40F6
:1022E00040F40000704700BF70B595B214460E462A
:1022F0002A464FF6FF73064801F0AAF82A463146EF
:102300004FF6FF73034801F0A3F8204670BD00BFED
:1023100090010020D0010020DFED187A184AB5EEB8
:10232000C00A20EE270AF1EE10FA70B501464FF010
:102330006405FDEEC07A0DD417EE903A82FB0302DD
:10234000DC17C4EB621205FB12330E48BDE8704087
:10235000FDF7FCBF17EE904A604282FB0036C317C0
:1023600082FB04E2C3EB6613E41705FB1303C4EB23
:1023700062120448BDE87040FDF7E8BF0000C842A3
:102380001F85EB51AC420108F0B595B008A830228A
:102390000021FDF777FF00241D4A01940494039463
:1023A000059406940794116C1A4B41F08051116406
:1023B000126C02F080520192019A02941A6842F45F
:1023C00080421A601B680F9403F480430293012338
:1023D0000225082148220B9308A8032310261091F8
:1023E00011921393029F08950E9512950C9601F089
:1023F00003FA0F224FF4805303A82946049505944D
:1024000007940392069301F0EDFB15B0F0BD00BFF9
:102410000038024000700040F0B5114C114A124BD8
:10242000226085B00025012607462046A36265602C
:102430000095A5602561A5612562E562E5602563DB
:10244000019502950395E661666100F00BFC694613
:10245000204600970196029500F078FD05B0F0BD8A
:1024600008010020002001400100000F38B50020C5
:102470002DED028BFFF7D0FF714800F0A7FC322151
:102480006F4800F00FFD6E4800F004FE810500F17A
:102490008A806C4B93ED000A6B48FFF73DFF0320E9
:1024A000FFF7BAFF664800F091FC3221644800F063
:1024B000F9FC634800F0EEFD820552D4634B93EDC6
:1024C000000A6348FFF728FF0420FFF7A5FF5C48D8
:1024D00000F07CFC32215A4800F0E4FC584800F03F
:1024E000D9FD83050DD45B4B93ED000A5A48FFF7E5
:1024F00013FFBDEC028B42F21070BDE8384001F0D2
:1025000037BE4F4800F01EFD83B207EE903ADFED74
:10251000536A9FED537A534A534B1080F8EEE77A93
:1025200067EEA67A67EE877AC3ED007A17EE900A17
:10253000FFF724FC4D4B044618680D46FFF71EFCC0
:1025400000224B4BFFF7BCFA0B46024629462046B9
:10255000FFF7B4FAFFF778FE3E4B00EE100A186062
:10256000C4E7374800F0EEFC83B207EE903ADFEDA7
:102570003B5A9FED3B6A3F4B9FED3F7AD3ED006A9C
:102580003E493F4A314B0880F8EEE77A67EEA57A7C
:1025900067EE867A27EE877AC2ED007A87EE260A02
:1025A00083ED000A8DE7264800F0CCFC83B208EEEC
:1025B000103A9FED2A7ADFED2A7A3249324AD1ED7C
:1025C000008A324B1080B8EEC88A28EE078A28EEBF
:1025D000278AB4EEE88AF1EE10FA83ED008A29DC4E
:1025E0002B4BD3ED007A78EEE77A17EE900AFFF7DF
:1025F000C5FB02460B4600202649FFF73DFD78EE5D
:10260000687A044617EE900A0D46FFF7B7FB0246BC
:102610000B4620462946FFF705FC0B4602461E499D
:102620000020FFF74BFAFFF70FFE064B00EE100AF3
:10263000186031E7194BD3ED007A77EEE87AD4E7EA
:1026400008010020C8000020B8420108D400002082
:10265000C0420108E0000020C84201083333534063
:1026600000008039DC000020E8000020E4000020A9
:102670000000F83F700000200000C842D000002099
:10268000D80000206C000020C4000020CC000020F6
:10269000640000200000084000001C40680000208A
:1026A000624B634A634C80B59A6001F039FDFFF7D5
:1026B0006BFE00F0DDF800F0D5F900F09BF900F0BA
:1026C000B5F90A2305225C495C4800F0C1FE4FF4CD
:1026D0007A7001F04DFD0A2305225949574800F050
:1026E000B7FE21464FF4FA631422544800F00CFF61
:1026F0000A2314222146534800F0AAFEA37C5A1E46
:10270000012A40F28B80052B05D10A230B224E496A
:102710004C4800F09DFE4D4E4D4D4E4C4E4FDFF857
:102720004881B3EE008A0DE0D5ED007AF4EEC87A68
:10273000F1EE10FA4AD4D4ED007AF4EEC87AF1EE54
:1027400010FA5AD4FFF792FED6ED007AF4EEC87A6A
:10275000F1EE10FAE8D500224FF400513F4801F0A5
:102760003FFC00224FF480713C4801F039FC00220C
:102770004FF400413A4801F033FC00224FF400517D
:10278000374801F02DFC00224FF40061344801F07D
:1027900027FC00224FF40041384601F021FC0022C2
:1027A0004FF40041404601F01BFC41F2883001F03B
:1027B000DFFC01224FF40051284801F011FCD5ED57
:1027C000007AF4EEC87AF1EE10FAB4D500224FF494
:1027D0000051234801F004FC41F2883001F0C8FCAC
:1027E00001224FF400511E4801F0FAFBD4ED007AAB
:1027F000F4EEC87AF1EE10FAA4D500224FF40041AD
:10280000384601F0EDFB41F2883001F0B1FC0122C5
:102810004FF40041384601F0E3FB93E70A23072217
:102820001049084800F014FE75E700BF00ED00E015
:1028300000000108F40000207C000020D0010020EE
:1028400074000020900100208C000020C8000020AF
:10285000D4000020E00000200004024000000240FC
:10286000000C02408400002000100240704700BFAE
:102870002DE9F0438BB00024464B00941A6B464D73
:10288000DFF82091DFF82081444F454E42F00102ED
:102890001A631A6B02F001020092009A01941A6BFB
:1028A00042F010021A631A6B02F010020192019AB0
:1028B00002941A6B42F002021A631A6B02F00202CF
:1028C0000292029A03941A6B42F008021A631A6B7E
:1028D00002F008020392039A04941A6B42F0040275
:1028E0001A631B6B03F004030493284601224FF480
:1028F0007841049B01F074FB484601224FF44041AB
:1029000001F06EFB404601224FF47C4101F068FB70
:10291000384601224FF4007101F062FB012230467B
:102920004FF47C5101F05CFB284605A901254FF4CA
:102930007843059307940894069501F03BFA4846BE
:1029400005A94FF44043059306950794089401F0B8
:1029500031FA404605A94FF47C4305930695079448
:10296000089401F027FA384605A94FF4007305933F
:1029700006950794089401F01DFA4FF47C5305A9BD
:102980003046069507940894059301F013FA0BB0AE
:10299000BDE8F08300380240001002400008024009
:1029A0000000024000040240000C024002680F4B8D
:1029B0009A4200D0704710B586B0002103F58C33E1
:1029C00000915A6C0A4842F480725A645B6C03911D
:1029D00003F4807300931022032301A9009C019249
:1029E000029301F0E7F906B010BD00BF00200140DE
:1029F000000002400B4B0C4A10B50C211A604FF43A
:102A0000E134002218465C6059619A60DA601A610C
:102A10009A61DA6100F0ECFC00B910BDBDE810402D
:102A2000FFF724BF90010020004C00400B4B0C4AE4
:102A300010B50C211A604FF4E134002218465C6096
:102A400059619A60DA601A619A61DA6100F0D0FC2B
:102A500000B910BDBDE81040FFF708BF50010020CD
:102A6000001001400B4B0C4A10B50C211A604FF4BA
:102A70001644002218465C6059619A60DA601A6157
:102A80009A61DA6100F0B4FC00B910BDBDE81040F5
:102A9000FFF7ECBED001002000440040F0B5036811
:102AA0003C4A934289B02BD03B4A93424DD03B4A9B
:102AB000934201D009B0F0BD0024394B0294196C47
:102AC000384841F4003119641B6C03F4003302935D
:102AD0000322072303A9602702260125DDF808E069
:102AE0000692079303970496059501F063F9224631
:102AF0002146262001F09CFA262001F0CFFAD9E7E2
:102B00000024274B0094196C274841F400211964D4
:102B10001B6C03F4002300930322082303A94FF442
:102B2000406702260125DDF800E00692079303972F
:102B30000496059501F03EF922462146342001F025
:102B400077FA342001F0AAFAB4E70024144B019478
:102B5000596C164841F0100159645B6C03F0100386
:102B600001930322072303A9C02702260125DDF8CC
:102B700004E00692079303970496059501F01AF96D
:102B800022462146252001F053FA252001F086FA3D
:102B900090E700BF004C004000100140004400409E
:102BA00000380240000C02400008024000040240CD
:102BB000704700BFFEE700BFFEE700BFFEE700BFB3
:102BC000FEE700BF704700BF704700BF704700BFFF
:102BD00008B501F0BFFABDE8084001F087BA00BFB0
:102BE000014800F03BBD00BF50010020014800F04B
:102BF00035BD00BFD0010020014800F02FBD00BF4F
:102C00009001002008B5032001F000FA00221146CF
:102C10006FF00B0001F00CFA002211466FF00A0071
:102C200001F006FA002211466FF0090001F000FAE7
:102C3000002211466FF0040001F0FAF9002211465B
:102C40006FF0030001F0F4F9002211466FF001006B
:102C500001F0EEF9002211464FF0FF30BDE80840C8
:102C600001F0E6B9002800F0AA80F8B5036C04462C
:102C70003BB1236CDB060CD50023012084F83C30EB
:102C8000F8BD436480F83C30FFF790FE236CDB0610
:102C9000F2D4226C4B4923684B4D22F4885222F027
:102CA000020242F0020222644A6822F440324A6080
:102CB0004A68606802434A6059682069D4F808E0AD
:102CC000E768A26A21F4807159605E6846EA0026CE
:102CD0005E605E6826F040765E60586840EA0E00EE
:102CE0005860986820F4006098609968AA4241EAA8
:102CF0000701996046D09968E06A21F07061996097
:102D000099680A439A60996821F0405199609A68DD
:102D100002439A609968A569206A21F002019960CE
:102D20009A6842EA45029A605A68002833D122F430
:102D300000625A60DA6AE569276B666922F47002FC
:102D4000DA62D86A013D40EA0550D862986820F4FA
:102D500000709860996841EA47219960996821F468
:102D6000806199609A68002042EA86229A606064D5
:102D7000236C23F0030343F001032364002384F84E
:102D80003C30F8BD9A6822F070629A609A6822F02E
:102D900040529A60BEE742F400625A605A6822F4D8
:102DA00060425A604FF4604191FAA1F1626A58683A
:102DB000B1FA81F1013A8A4002435A60BAE7012030
:102DC000704700BF002301400100000F10B490F8CD
:102DD0003C3083B00022012B019255D002689368E9
:102DE0000121DB0780F83C1014D42A4B2A4C1B68C5
:102DF0009168A4FB03439B0C03EB430341F00101E7
:102E000091600193019B2BB1019B013B0193019BBD
:102E1000002BF9D19368DC0731D5036C23F4E06310
:102E200023F0010343F4807303645368590505D507
:102E3000036C23F4405343F480530364036C13F492
:102E400080531CBF436C23F00603436400246FF0DF
:102E50002201124B80F83C4011605B68DB060BD10D
:102E6000906810F040500AD1936843F0804393601B
:102E700003B05DF8044B7047094B9A42F0D0002034
:102E800003B05DF8044B7047022003B05DF8044BBB
:102E9000704700BF9800002083DE1B4300230140E1
:102EA0000020014003689A68520502D59B68DB0543
:102EB0003ED470B50C46054601F054F906462A6822
:102EC00001E0601C25D113689907FAD56FF0120351
:102ED00013602B6C43F400732B64936813F0405F12
:102EE00015D1AB699BB9D36A13F4700F0CD12B6C5D
:102EF00023F480732B64286C10F4805007D12B6C62
:102F000043F001032B6470BD93685B05EFD500208F
:102F100070BD24B101F026F9801B8442CFD22B6C06
:102F2000002243F004032B6485F83C20032070BD8D
:102F3000036C002243F02003036480F83C2001204E
:102F4000704700BF0368D86C704700BFF0B590F8B9
:102F50003C3083B00022012B019257D00D68012331
:102F6000092D2E4680F83C3029D804688B682269E8
:102F700005EB450E072707FA0EF722EA0702226142
:102F8000226903FA0EF3134323614B68062B2BD8F7
:102F900003EB8303626B053B1F21994022EA010288
:102FA0006263626B06FA03F313436363364B9C421E
:102FB0003ED0002380F83C30184603B0F0BD0468D2
:102FC0008B68E768AEB206EB46021E3A4FF0070E7A
:102FD0000EFA02FE27EA0E07E760E76893403B43DC
:102FE000E3604B68062BD3D90C2B12D803EB830379
:102FF000A3F123011F22236B8A4023EA02032363E8
:10300000236B06FA01F119432163CFE7022003B0D5
:10301000F0BD03EB8302413AE36A1F21914023EAAA
:103020000103E362E36A06FA02F11943E162BDE7D4
:10303000122D23D0A5F11003012BBAD8134A5368DF
:10304000102D43F400035360B3D1114B02F14672CB
:1030500002F52E321B6802F28332A2FB03239B0C83
:1030600003EB83035B000193019B002BA1D0019B29
:10307000013B0193019B002BF9D19AE7034A536866
:1030800043F48003536094E7002001400023014093
:1030900098000020006C70472DE9F0470468226911
:1030A0008246C068DAF81C10DAF80830DAF81060E6
:1030B000DAF8145022F4405202432261E268DAF84E
:1030C0001800334322F416422B4322F00C020B4328
:1030D0001343E360636923F440730343B1F5004F86
:1030E0006361AB4B61D09C4200F0018103F58063CA
:1030F0009C4200F0FC8000F02DFEA64FDAF8043070
:1031000000EB800000EB80009B00B0FBF3F3A7FB1B
:1031100003235B091D0100F01DFEDAF8043000EB0B
:1031200080009B0000EB8000B0FBF3F600F012FE85
:10313000DAF8042000EB8000930000EB8000B0FB85
:10314000F3F3A7FB03234FF064095B0909FB136347
:103150001B013233A7FB03235B0903F0F00600F0E9
:10316000F9FDDAF8042000EB8000930000EB80000A
:10317000B0FBF3F800F0EEFDDAF8043000EB80006D
:103180009B0000EB8000B0FBF3F0A7FB0030400990
:1031900009FB10831B013233A7FB0323C3F3431343
:1031A00033432B44A360BDE8F0879C425DD003F518
:1031B00080639C4259D000F0CDFD764FDAF80430A0
:1031C00000EB800000EB80005B00B0FBF3F3A7FB9B
:1031D00003235B091E0100F0BDFDDAF8043000EBAB
:1031E00080005B0000EB8000B0FBF3F500F0B2FD67
:1031F000DAF8042000EB8000530000EB8000B0FB05
:10320000F3F3A7FB03235B094FF0640909FB135396
:10321000DB003233A7FB03231B0903F4F87500F02E
:1032200099FDDAF8042000EB800000EB80005300E9
:10323000B0FBF3F800F08EFDDAF8043000EB80000C
:1032400000EB80005B00B0FBF3F3A7FB03235B09FB
:1032500009FB1383DB003233A7FB0323C3F34213C1
:1032600033442B44A360BDE8F08700F08BFD494F49
:10327000DAF8043000EB800000EB80005B00B0FB6C
:10328000F3F3A7FB03235B091E0100F07BFDDAF8D3
:10329000043000EB80005B0000EB8000B0FBF3F536
:1032A00000F070FDDAF8042000EB8000530000EB22
:1032B0008000B0FBF3F3A7FB03234FF064095B0925
:1032C00009FB1353DB003233A7FB03231B0903F471
:1032D000F87500F057FDDAF8042000EB8000530089
:1032E00000EB8000B0FBF3F800F04CFDA4E700F029
:1032F00049FD284FDAF8043000EB800000EB800035
:103300009B00B0FBF3F3A7FB03235B091D0100F057
:1033100039FDDAF8043000EB80009B0000EB800000
:10332000B0FBF3F600F02EFDDAF8042000EB80008D
:10333000930000EB8000B0FBF3F3A7FB03234FF0F7
:1033400064095B0909FB13631B013233A7FB0323E9
:103350005B0903F0F00600F015FDDAF8042000EB3D
:103360008000930000EB8000B0FBF3F800F00AFD52
:10337000DAF8043000EB800000EB80009B00B0FB2B
:10338000F3F3A7FB03235B0909FB138302E700BFE9
:10339000001001401F85EB512DE9F04107460E4614
:1033A00090461D463C6801E06B1C06D1206836EA59
:1033B0000003F9D10020BDE8F08135B100F0D2FE64
:1033C000A0EB08008542EDD23C68E36823F4D0739B
:1033D000E3606369202223F001030021636103207D
:1033E00087F8392087F8381087F83A20BDE8F0814F
:1033F00060B338B590F83930044603F0FF0203B3E8
:103400002268242384F83930D36823F40053D3602E
:103410002046FFF741FE23681A6922F490421A61A0
:103420005A6922F02A025A61DA680025202142F402
:103430000052DA602846E56384F8391084F83A10BF
:1034400038BD80F83820FFF729FBD9E70120704705
:103450002DE9F0430F4690F83910202983B003D0AE
:10346000022003B0BDE8F083002F3ED0002A3CD0FC
:10347000984690F83830012B0446F1D00020012105
:103480002123E06384F8381084F83930019200F089
:1034900069FE019AA2848146E28406E0FFF77CFF80
:1034A00028BB23683A785A600137E58CADB24346B1
:1034B0004A4680212046E5B1E58CA668013DADB2C3
:1034C000B6F5805FE584E9D143464A46802120462F
:1034D000FFF762FF58B93B8821682269C3F30803EC
:1034E0004B60002AE0D10237DFE70120B9E7032073
:1034F000B7E74021FFF750FF0028F8D1202384F8D8
:10350000380084F83930ACE72DE9F0430E4690F8E6
:103510003A10202983B003D0022003B0BDE8F08325
:1035200076B36AB3984690F83830012B0446F3D04E
:10353000002001212223E06384F8381084F83A3017
:10354000019200F00FFE019AA2858146E285E58D89
:10355000ADB243464A462021204685B3E58DA76893
:10356000013DADB2B7F5805FE58512D0FFF714FFDE
:1035700058BB236933B923685B6833700136E6E7CB
:103580000120CAE723685B6803F07F0333700136CC
:10359000DDE743464A4620212046FFF7FDFEA0B95D
:1035A000236933B923685B68C3F3080326F8023B39
:1035B000CDE723685B68DBB226F8013BC7E784F8F8
:1035C0003850284684F83A10A7E70320A5E700BF43
:1035D000704700BF704700BF8368B3F5805F28D095
:1035E000036973B10368826A5B68511C03F07F034F
:1035F00081621370C38D013B9BB2C38543B1002030
:103600007047836A0268591C526881621A70F1E738
:103610000268D16821F4907110B5D16051692024FD
:1036200021F00101516180F83A40FFF7D3FF0020FB
:1036300010BD0269836A3AB902685268C2F308028F
:1036400023F8022B8362D5E702685268D2B223F8CE
:10365000012B8362CEE700BF704700BF03681A6882
:1036600070B51607DD685969044649D011F00101AB
:1036700052D0D60705D5E80503D5E06B40F0010030
:10368000E06356077AD5002900F08480E16B90074B
:1036900041F00201E16376D5E16B41F00401E163A1
:1036A000110772D4E16B002929D0910605D5AA062D
:1036B00003D594F83A20222A7CD05D69E16B0E078D
:1036C00002D415F040057AD0DA6822F49072DA60FC
:1036D0005A69202122F001025A6184F83A105A698D
:1036E00055065ED55A69606B22F040025A61002887
:1036F00057D03B4B036500F077FC002855D170BDD7
:1037000096060CD5A9060AD590F83A30222BF6D1A8
:10371000BDE87040FFF760BF15F4907FA9D1100697
:103720000ED45606EBD56D06E9D5DA68202122F0D5
:103730004002DA60204684F83910FFF749FF70BD77
:103740002906EED594F83920212AD8D1A268B2F5FD
:10375000805F226A38D0511C216212785A60E28C54
:10376000013A92B2E284002AC9D1DA6822F08002DA
:10377000DA60DA6842F04002DA6070BD96070BD575
:10378000002989D18EE711078CD5E16B41F0080142
:10379000E16387E7900785D4100783D5002981D09E
:1037A000F3E72046FFF758FF70BD606BBDE870403F
:1037B000036D18472046FFF70FFF23687DE720467B
:1037C000FFF74AFFE56370BD11882069C1F3080166
:1037D000596010B902322262C1E701322262BEE7AB
:1037E000E537010808B5836B0022DA851846DA84CC
:1037F000FFF732FF08BD00BFF0B50368DD0783B0F7
:1038000004462FD5A3498A6802F00C02042A00F06E
:10381000F4808A6802F00C02082A00F0EA806368EB
:10382000B3F5803F00F02C81B3F5A02F00F00081AC
:10383000984D2A6822F480322A602A6822F4802275
:103840002A60002B40F0FD8000F08CFC064605E06D
:1038500000F088FC801B642800F2AA802B689B0380
:10386000F6D423689F072DD58A4A916811F00C0F72
:1038700000F0A580916801F00C01082900F09B8000
:10388000E368002B00F0EB80834B824D01221A602D
:1038900000F068FC064605E000F064FC801B02288E
:1038A00000F286802B689807F6D52968F82292FAEC
:1038B000A2F22369B2FA82F221F0F80193400B439D
:1038C0002B6023681A0720D4590734D4A369CBB1DD
:1038D000704DAA6802F00C02082A77D0022B6F4BB9
:1038E0004FF000021A6000F0D18000F03BFC2C4643
:1038F000054604E000F036FC401B022858D8236837
:103900009B01F7D4002003B0F0BD6369002B60D0A9
:10391000634B604D01221A6000F024FC064604E06F
:1039200000F020FC801B022842D86B6F9F07F7D560
:1039300023685907CAD5574B5A4D002201921A6C79
:1039400042F080521A641B6C03F080530193019B78
:103950002B6843F480732B6000F004FC064604E0FF
:1039600000F000FC801B022822D82B68DA05F7D56E
:10397000A368012B00F0F180052B00F0D580454DA8
:103980002A6F22F001022A672A6F22F004022A67B6
:10399000002B40F0D28000F0E5FB41F2883607466C
:1039A0002B6F980792D500F0DDFBC01BB042F7D912
:1039B000032003B0F0BD526856023FF561AF354AAF
:1039C0001268950723D5E268012A20D0012003B0B0
:1039D000F0BD334A2F4D136000F0C4FB064604E0EF
:1039E00000F0C0FB801B0228E2D86B6F9807F7D469
:1039F0009EE74A6850027FF512AF264A126891038B
:103A00007FF530AF6268002A7FF42CAFDEE7214DEE
:103A1000F821286891FAA1F12269B1FA81F120F028
:103A2000F8008A4002432A601A077FF54DAF6CE721
:103A3000184B1A6842F480221A601A6842F48032E5
:103A40001A6000F08FFB134D064604E000F08AFB7D
:103A5000801B6428ACD82B689A03F7D501E70E4A7F
:103A60000C4D136000F07EFB064604E000F07AFB8C
:103A7000801B02289CD82B689907F7D4236821E77C
:103A8000044A136843F480331360DAE700F06AFBFA
:103A900006460FE0003802400000474260004742FF
:103AA000800E47420070004000F05CFB801B022843
:103AB0003FF67EAF2B689901F6D447F6C07696FAAA
:103AC000A6F64FF44032B6FA86F692FAA2F24FF01A
:103AD0007061B2FA82F091FAA1F1A26A676AE369B1
:103AE000D4F820E0E46A520843EA0E0307FA06F627
:103AF000013A8240B1FA81F1334304FA01F11343F0
:103B0000194A1A4C0B4301216B60116000F02AFB2B
:103B1000054605E000F026FB401B02283FF648AFB3
:103B200023689A01F6D5EDE6104B1A6F42F00402B5
:103B30001A671A6F42F001021A6700F013FB0B4D6F
:103B4000074641F288362B6F9B073FF5BFAE00F06A
:103B500009FBC01BB042F6D92AE7044A136F43F0B1
:103B600001031367E9E700BF6000474200380240E5
:103B7000194A936803F00C03042B2BD0082B27D190
:103B80005168536801F03F0113F4800F536847F602
:103B9000C07292FAA2F0B0FA80F003EA020323FAAC
:103BA00000F314BF0D480E48B0FBF1F000FB03F02A
:103BB000094B4FF440325B6892FAA2F2B2FA82F2F9
:103BC00003F44033D34001335B00B0FBF3F07047A4
:103BD00003487047014870470038024040787D0133
:103BE0000024F400574A136803F00F038B4208D2F5
:103BF000CBB21370136803F00F03994201D0012078
:103C0000704703689A072DE9F04106D54E4C856848
:103C1000A26822F0F0022A43A260DF0706460C46A3
:103C200026D54268012A00F08780931E012B464B5F
:103C30001B687BD9990728D5434DAB6823F0030354
:103C40001343AB6000F08EFA7368012B074641F214
:103C500088384FD0022B58D0032B05D160E000F0FC
:103C600081FAC01B404564D8AB6813F00C0FF6D145
:103C7000344A136803F00F039C4209D2E3B2137075
:103C8000136803F00F039C4202D00120BDE8F081CD
:103C900033685A0706D52C49F0688A6822F4E05246
:103CA00002438A601B0707D5274A3169936823F4CA
:103CB000604343EAC1039360FFF75AFF224B01467A
:103CC000F0229B6892FAA2F2B2FA82F203F0F003B9
:103CD000D3401E481E4AC35C002021FA03F3136040
:103CE00000F008FA0020BDE8F08100F03BFAC01BAC
:103CF00040451ED8AB6803F00C03042BF5D1B7E7A1
:103D000000F030FAC01B404513D8AB6803F00C0339
:103D1000082BF5D1ACE700F025FAC01B404508D8C8
:103D2000AB6803F00C030C2BF5D1A1E7980183D409
:103D3000ABE70320BDE8F081034B1B689D033FF513
:103D40007BAFA2E7003C024000380240D0420108AD
:103D500098000020084B4FF4E0529B6892FAA2F2C0
:103D6000B2FA82F203F4E053D3400449044ACB5C34
:103D70001068D840704700BF00380240D0420108A8
:103D800098000020084B4FF460429B6892FAA2F220
:103D9000B2FA82F203F46043D3400449044ACB5C94
:103DA0001068D840704700BF00380240D042010878
:103DB000980000202DE9F04FD1F800C0DFF8148200
:103DC000DFF814E283B0002503E00135102D00F088
:103DD0009B800123AB4003EA0C029342F5D14E686D
:103DE00026F0100ABAF1020F00F091804FEA45095F
:103DF0000324D0F800B004FA09F4E44306F0030702
:103E00000BEA040B07FA09F70AF1FF3A47EA0B0736
:103E1000BAF1010F076040F2A080C7688B683C4090
:103E200003FA09F32343C360F300CED54FF0000932
:103E3000CDF80490D8F8443043F48043C8F84430B7
:103E4000D8F8444025F0030303F1804304F4804490
:103E500003F59C33019405F00304019FD3F808A0F7
:103E6000A4000F27A7402AEA070A544FB84222D0DD
:103E700007F58067B84200F08380514FB84200F0E8
:103E80008480504FB84200F085804F4FB84200F018
:103E900086804E4FB84200F087804D4FB84200F008
:103EA0008880DFF8389148450CBF4FF007094FF084
:103EB000080909FA04F94AEA09079F60DEF80030A8
:103EC000D443F70354BF23401343CEF80030DEF849
:103ED0000430B70354BF23401343CEF80430DEF858
:103EE0000830F70254BF23401343CEF80830DEF801
:103EF0000C30B60205F1010554BF23401343102DC9
:103F0000CEF80C307FF465AF03B0BDE8F08F4FEA18
:103F1000D50900EB890905F00707D9F82040BF0053
:103F20004FF00F0B0BFA07FB24EA0B0A0C69BC409D
:103F300044EA0A04C9F820404FEA45090324D0F8AE
:103F400000A004FA09F4E44306F003070AEA040AAD
:103F500007FA09F747EA0A070760876807EA040AC9
:103F6000CF6807FA09F747EA0A078760D0F804A084
:103F7000C6F300172AEA0303AF401F4347604CE72C
:103F80004FF0010909FA04F995E74FF0020909FA1F
:103F900004F990E74FF0030909FA04F98BE74FF0B1
:103FA000040909FA04F986E74FF0050909FA04F94A
:103FB00081E74FF0060909FA04F97CE700000240A6
:103FC00000080240000C02400010024000140240B1
:103FD0000018024000380240003C0140001C024032
:103FE00002B909048161704790F83530022B03D083
:103FF00080234365012070470268052380F835302F
:10400000136823F00103136000207047074AD36848
:104010004FF6FF010B40000243F0BF6300F4E06085
:1040200043F400330343D360704700BF00ED00E06A
:10403000184B70B4DC68C4F30224C4F10706042EE4
:1040400004F1040328BF0426062B17D9033C0125DD
:10405000A540013D2A400123B340013B1940A14046
:10406000002841EA02010CDB00F1604000F56140EC
:104070000901C9B280F8001370BC704700221446D1
:10408000E9E7054B00F00F0009010344C9B21976B6
:1040900070BC704700ED00E0FCEC00E000F01F0198
:1040A00001234009024A8B4042F82030704700BF8C
:1040B00000E100E00138B0F1807F0ED2084B10B46F
:1040C000084C5860F02084F8230000220721104695
:1040D0009A6019605DF8044B70470120704700BF7B
:1040E00010E000E000ED00E0704700BF08B5FFF70A
:1040F000FBFF08BD084B094A1B6810B5A2FB032350
:1041000004469809FFF7D6FF214600224FF0FF3002
:10411000FFF78EFF002010BD98000020D34D6210E5
:1041200008B50B4B1A6842F400721A601A6842F420
:1041300080621A601A6842F480721A600320FFF7E6
:1041400065FF0020FFF7D6FFFEF75CFD002008BDED
:10415000003C0240024A136801331360704700BFFD
:1041600010020020014B1868704700BF10020020A9
:1041700010B582B00190FFF7F5FF0446FFF7F2FF9C
:10418000019B001B9842F9D302B010BD1049114B9E
:10419000D1F8882042F4700210B4C1F888201A685F
:1041A0000D4C002042F001021A6098601A6822F05B
:1041B000847222F480321A605C601A684FF00064E6
:1041C00022F480221A60D8608C605DF8044B70473E
:1041D00000ED00E00038024010300024DFF834D059
:1041E000002103E00C4B5B58435004310B480C4B4F
:1041F00042189A42F6D30B4A02E0002342F8043BED
:10420000094B9A42F9D3FFF7C1FFFCF713F8FEF709
:1042100047FA7047000002202843010800000020F0
:104220009C0000209C00002018020020FEE70000F7
:10423000F8B500BFF8BC08BC9E467047F8B500BF93
:08424000F8BC08BC9E46704763
:104248000400002000000000000000000000000042
:104258000000000000000000000000000000000056
:104268000000000000000000000000000000000046
:104278000000000000000000000000000000000036
:104288000000000000000000000000000000000026
:104298000000000000000000000000000000000016
:1042A800000000002573203D2025642E25640A00A7
:1042B8004D345F50480000004D355F444F0000000A
:1042C8004D375F4F52500000000000000102030408
:1042D800010203040607080943000000232D302BC0
:1042E80020000000686C4C00656667454647000082
:1042F8003031323334353637383941424344454614
:1043080000000000303132333435363738396162D5
:0843180063646566000000000B
:04432000FD01010892
:04432400D5010108B6
:1043280004000020000000008C4201086C420108D3
:104338004C420108000000000000000000000000DE
:1043480000000000E042010800000000000000003A
:104358000000000000000000000000000000000055
:104368000000000000000000000000000000000045
:104378000000000000000000000000000000000035
:10438800000000009A99793F85EB01400000C03F8A
:10439800AE47E13EFE00010001000000FE00020001
:1043A80002000000636F6E6E656374006E6F7420A8
:0C43B800636F6E6E656374000024F400F7
:04000005080141DDD0
:00000001FF
